:020000040800F2
:100000006025002095020008A32700084921000868
:10001000A1270008D10A0008392D000800000000BF
:10002000000000000000000000000000FD010008CA
:100030000B0B000800000000410200082F290008F7
:10004000AF020008AF020008AF020008AF020008CC
:10005000AF020008AF020008AF020008AF020008BC
:10006000AF020008AF020008AF020008AF020008AC
:10007000AF020008D50A0008AF020008AF0200086E
:10008000AF020008AF020008AF020008AF0200088C
:10009000AF020008AF020008AF020008AF0200087C
:1000A000AF020008AF020008AF020008AF0200086C
:1000B000AF020008AF020008AF020008AF0200085C
:1000C000AF020008AF020008AF020008AF0200084C
:1000D000AF020008AF020008AF020008AF0200083C
:1000E000AF020008AF020008AF02000800000000E5
:1000F0000000000000000000000000000000000000
:100100000000000000000000AF020008AF0200087D
:10011000AF020008AF020008AF020008AF020008FB
:10012000AF020008AF020008AF020008AF020008EB
:10013000AF0200080000000000000000AF0200084D
:10014000AF020008AF020008AF020008AF020008CB
:1001500000F002F800F043F80AA090E8000C824496
:100160008344AAF10107DA4501D100F038F8AFF273
:10017000090EBAE80F0013F0010F18BFFB1A43F085
:1001800001031847704E0000904E0000103A24BF43
:1001900078C878C1FAD8520724BF30C830C144BFEC
:1001A00004680C607047000000230024002500262E
:1001B000103A28BF78C1FBD8520728BF30C148BFCA
:1001C0000B607047752900F06781002070471FB5EC
:1001D0009DE8030000F08CFA1FBD10B510BD00F0C3
:1001E000AFFB1146FFF7F3FF02F0F2FD00F0CDFB8D
:1001F00003B4FFF7F2FF03BC00F0FEFB224B1968CB
:100200000868B0E8F00F80F30988BFF36F8F4FF0F4
:10021000000080F311884EF00D0E704700000000C2
:1002200006480068006880F3088862B661B6BFF3CC
:100230004F8FBFF36F8F00DF00BF00BF08ED00E0FE
:10024000EFF30980BFF36F8F0F4B1A6820E9F00FAF
:10025000106008B54FF0500080F31188BFF34F8F46
:10026000BFF36F8F03F04CFD4FF0000080F3118857
:10027000BDE8084019680868B0E8F00F80F3098805
:10028000BFF36F8F704700BF1C000020EFF30580A5
:10029000704700000948804709480047FEE7FEE72D
:1002A000FEE7FEE7FEE7FEE7FEE7FEE7FEE7FEE726
:1002B00004480549054A064B70470000B12900086B
:1002C00051010008601F00206025002060210020EF
:1002D0006021002070B5064600F0EEF9056806F1D1
:1002E0000B0020F00704B4429CBF002070BD2B46D9
:1002F0006A68BAB11068A04210D304F108018842BC
:100300003CBF5068586007D35168101941601168AC
:10031000091B016058601460101D70BD13465268BF
:10032000002AE7D12146284600F0CEF90028DED188
:1003300070BD70B50446051F00F0BEF90068002CC2
:1003400014BF446870BD002C18BFAC423CBF2046AF
:100350006468F8D301680A18AA4218BF456003D13F
:100360002A6805461144016028684119A1421CBF52
:100370006C6070BD6168696021680844286070BD68
:1003800053EA020C00F069802DE9F04B4FF00006B3
:10039000002B1FBFB3FA83F503FA05F424FA05F620
:1003A0005E4012BF1643B2FA82F502FA05F4C5F1B7
:1003B00020051EBF22FA05FC44EA0C04203556EA4B
:1003C000044C4FEA144418BF641C4FF000084FF06F
:1003D0000009904271EB030C39D3002919BFB1FA1F
:1003E00081F701FA07F6B0FA80F700FA07F6C7F1CD
:1003F00020071EBF20FA07FC46EA0C062037B6FB92
:10040000F4FCA7EB0507103F07F01F0BCBF120060C
:100410000CFA0BFB2CFA06F644BFB3460026202F3D
:10042000A4BF5E464FF0000B5BEA060C08BF4FF01E
:10043000010B19EB0B09ABFB027C48EB0608C01B58
:1004400006FB02CC0BFB03CC71EB0C01C1E70B46A6
:10045000024641464846BDE8F08B13B54FF0000018
:100460004FF00001AFF30080BDE81C407047000072
:100470000FB41CB5074B06AA7B446946009005984B
:1004800000F0CBF90020694600F0DAF91CBC5DF8F9
:1004900014FB0000C50300002DE9F04106460024CE
:1004A00010687529314616A510D0AFF300800028DA
:1004B00002DA404213A507E031688A0701D512A588
:1004C00002E0490704D511A5012401E0AFF3008043
:1004D00000210A2206F1240709E0B0FBF2FCB0FB80
:1004E000F2F302FB1C00303078541846491C0028F7
:1004F000F3D123462A463046BDE8F04100F02EB93C
:10050000000000002D0000002B0000002000000073
:100510002DE9F0410F460546002028622846E9688B
:10052000884770B3252805D0D5E901219047286A6E
:10053000401CF2E7E9682846002688476C280446F4
:100540000AD0682C08D04C2C35D06A2C31D0742CB1
:1005500031D07A2C2FD016E0E96806462846884725
:10056000B042044608D16C2E23D04FF48066284652
:10057000E9688847044606E06C2E03D04FF4807685
:1005800001E01EE04026E4B1A4F14100192802D8A0
:10059000203446F400663A46214628462E60FFF78E
:1005A00011FE60B1012808D0FF1D27F007070837AA
:1005B000B4E78026DBE70026D9E73F1DAEE72046FB
:1005C000B2E7286ABDE8F081032A40F2308010F0DB
:1005D000030C00F0158011F8013BBCF1020F6244DE
:1005E00098BF11F801CB00F8013B38BF11F8013B6F
:1005F000A2F1040298BF00F801CB38BF00F8013B1C
:1006000011F0030300F02181083AC0F0088051F88E
:10061000043B083A51F804CBA0E80810F5E7121D96
:100620005CBF51F8043B40F8043BAFF30080D207B5
:1006300024BF11F8013B11F801CB48BF11F8012B81
:1006400024BF00F8013B00F801CB48BF00F8012BA4
:10065000704702F0FF0343EA032242EA024200F03D
:1006600028B94FF0000200B513469446964620394B
:1006700022BFA0E80C50A0E80C50B1F12001BFF45B
:10068000F7AF090728BFA0E80C5048BF0CC05DF8C1
:1006900004EB890028BF40F8042B08BF704748BF0F
:1006A00020F8022B11F0804F18BF00F8012B704783
:1006B000704770477047000000487047081F0020CF
:1006C000704770477047704738B504460A460020A7
:1006D0006946AFF30080002808BF38BD0246009984
:1006E000204600F00BF9012038BD012000F020B9B0
:1006F000F8B5AFF30080054600200C46102000BF7F
:100700000646A819A0420DD9324669460020AFF32B
:100710000080070008BF00F00BF90098A04218BF46
:100720000546C419FFF7C8FF05600746F01D20F015
:1007300007004619284600F00AF8B44208BFF8BD81
:10074000A21B31463868BDE8F84000F0D7B8002158
:100750000160C0E901107047102070472DE9F04793
:100760000D4699469246044600F124080168880621
:1007700004D5E06921F01001216000E00120A842C9
:1007800001DD471B00E00027A1697A1902EB09008F
:10079000081AA0612078C00602D42046AFF300807A
:1007A000002608E0D4E901211AF806009047206AE3
:1007B000401C761C20624E45F4DB2078C0060AD52A
:1007C0002046AFF3008006E0D4E9012130209047B5
:1007D000206A401C2062381EA7F10107F4DC07E004
:1007E000D4E9012118F805009047206A401C2062D6
:1007F000281EA5F10105F3DC2046AFF30080207828
:10080000000602D50220BDE8F0870120FBE70000CA
:1008100001694A1C02610878704700B58FB0CDE9C4
:1008200001310021059105497944CDE903101146B4
:100830006846FFF76DFE0FB000BD0000E5FFFFFF4B
:100840000A6802F8010B0A60704710B5203AC0F040
:100850000B80B1E81850203AA0E81850B1E81850C1
:10086000A0E81850BFF4F5AF5FEA027C24BFB1E8FE
:100870001850A0E8185044BF18C918C0BDE810406F
:100880005FEA827C24BF51F8043B40F8043B08BF78
:100890007047D20728BF31F8023B48BF11F8012B3F
:1008A00028BF20F8023B48BF00F8012B70474FF0EB
:1008B00000020429C0F0128010F0030C3FF4D3AE04
:1008C000CCF1040CBCF1020F18BF00F8012BA8BF3B
:1008D00020F8022BA1EB0C01FFF7C5BE5FEAC17C3B
:1008E00024BF00F8012B00F8012B48BF00F8012BB2
:1008F0007047000000487047001F00200346406812
:100900008C46002818BF88423CBF03464068F8D395
:1009100018681844884207D00CF1030020F0070043
:10092000001D411A521A0146081D0A60FFF701BD59
:1009300010B500F039F8BDE8104000F02FB870474E
:100940007546FFF7D7FFAE4605006946534620F0CF
:100950000700854618B020B5FFF7AAFCBDE8204087
:100960004FF000064FF000074FF000084FF0000B6B
:1009700021F00701AC46ACE8C009ACE8C009ACE81E
:10098000C009ACE8C0098D46704710B50446AFF306
:1009900000802046BDE81040FFF72ABC002801D0A7
:1009A00000F02AB87047000010B5012805D00021DA
:1009B00003A000F027F8012010BD09A1F8E700000E
:1009C00053494752544D454D3A204F7574206F6638
:1009D0002068656170206D656D6F727900000000A0
:1009E0003A2048656170206D656D6F727920636F84
:1009F000727275707465640001491820ABBEFEE721
:100A00002600020070B505460C460A2000E06D1C69
:100A100000F011F835B128780028F8D102E0641C04
:100A200000F009F814B120780028F8D1BDE8704032
:100A30000A20AFF3008008B569468DF80000032056
:100A4000ABBE08BD2DE9F04105464FF07E500E4685
:100A50004FF0FF37824220DC114603F0B5FF194901
:100A600003F0E6FE03F0C4FE82B21748006825B129
:100A7000012D05D0022D10D105E00021426304E0D4
:100A80000421826301E00821C2630124AC400F4DC0
:100A900086B1012E07D0022E02D03846BDE8F08183
:100AA0002868044206D0084801F0A0FA2868A0434C
:100AB000286005E0044801F045FA286804432C60EA
:100AC0000020EBE700FF7F478C0100209C00002006
:100AD000FEE70000014800F017B9000048010020BF
:100AE00030B590F840500124AC40C56B6C60046890
:100AF00063604368102B036803D099600068C2608C
:100B000030BD9A600068C16030BD704772B6FEE7C4
:100B100070B5040003D094F8200010B104E0012067
:100B200070BD204600F082F82068016841F00101A4
:100B3000016000F08BFB0546052604E000F086FB13
:100B4000401B0A2811D820684068C007F6D02068EA
:100B5000016821F00201016000F078FB05460BE01E
:100B600000F074FB401B0A2806D9606A40F400308C
:100B7000606284F82060D2E7206840688007EFD484
:100B8000207E0128206801683DD021F080010160AD
:100B9000607E01282068016838D021F040010160A2
:100BA000A07E01282068016833D021F02001016077
:100BB000E07E0128206801682ED041F0100101601C
:100BC000207F01282068016829D021F008010160F8
:100BD000607F01282068016824D021F004010160B1
:100BE000D4E902010843D4E90412114308436168BF
:100BF000491E08432168C86100206062012084F812
:100C00002000002070BD41F08001C0E741F04001AC
:100C1000C5E741F02001CAE721F01001CFE741F01C
:100C20000801D4E741F00401D9E70000F0B585B030
:100C30000021304A00910191029103912C4F1168DB
:100C40000368BC14022503262B48491CBB4220D153
:100C50001160012907D1C16941F00071C161C16909
:100C600001F000710491816941F0040181618069A2
:100C7000224F00F0040004904FF400600090694699
:100C8000384600F0EDF9694638460396CDE900454F
:100C900029E01B4FBB4228D1C36943F08063C36185
:100CA000C369012903F080630493116007D1C1690E
:100CB00041F00071C161C16901F000710491816965
:100CC00041F0080181618069009400F008000D4C3A
:100CD00004906946204600F0C3F96014CDE9000590
:100CE00069460396204600F0BBF905B0F0BD000050
:100CF000006400400800002000100240000801408D
:100D000000680040000C01402DE9F05FC16B0A68EB
:100D100001680B68046C4FF0040808FA04F8844D6D
:100D2000844E854FDFF814C2DFF81492DFF814A266
:100D3000DFF814B2DFF814E218EA020F65D05FEAB8
:100D4000437862D50A68920603D40A6822F0040246
:100D50000A60DFF8F0814FF48062016808F114083E
:100D600013011402414524D9A9420DD0B1420FD03C
:100D7000B9421AD0614515D0494515D0514501D128
:100D8000120312E0594501D104220EE0714501D150
:100D900040220AE06D4D1435A94206D06B4A283234
:100DA000914201D11A4600E022466749091F0A60B4
:100DB00029E0A94213D0B14215D0B94220D06145F3
:100DC0001BD049451BD0514502D14FF4800217E09A
:100DD000414502D14FF0806212E0594501D1042211
:100DE0000EE0714501D140220AE0584D1435A94268
:100DF00006D0564A2832914201D11A4600E02246D6
:100E00004B4908394A60C16A71E04FF0020808FA9C
:100E100004F818EA020F70D05FEA83786DD50A688B
:100E2000920606D40A6822F00A020A60012180F8BC
:100E30002110DFF810814FF40072016808F11408E6
:100E400013011402414524D9A9420DD0B1420FD05B
:100E5000B9421AD0614515D0494515D0514501D147
:100E6000120312E0594501D102220EE0714501D171
:100E700020220AE0354D1435A94206D0334A2832E3
:100E8000914201D11A4600E022462F49091F0A600B
:100E900029E0A94213D0B14215D0B94220D0614512
:100EA0001BD049451BD0514502D14FF4001217E029
:100EB000414502D14FF0007212E0594501D10222A2
:100EC0000EE0714501D120220AE0204D1435A942DF
:100ED00006D01E4A2832914201D11A4600E022462D
:100EE000134908394A60002180F82010816A0029DE
:100EF0001CD0BDE8F05F0847FFE70825A540154274
:100F000014D01A0712D50A6822F00E020A6090F86F
:100F10004020C36B012101FA02F25A60816380F81C
:100F20002110002180F82010016BE0E7BDE8F09F60
:100F3000080002401C000240300002404400024011
:100F4000580002406C000240080402401C040240A9
:100F500030B560B11A4B026814219A4209D2194B7C
:100F60001344B3FBF1F18900016417490AE0012041
:100F700030BD134B5B421344B3FBF1F189000164B4
:100F80000F490839C163022180F82110136843F624
:100F9000F0718B43F0E901142143D0E902452C4361
:100FA000214304692143446921438469214319434E
:100FB000116000214163012242770177084630BD6C
:100FC00008040240F8FFFDBF0000024070B504466F
:100FD00090F82000002501280CD0012084F8200082
:100FE00094F821600020012E06D084F8200002250C
:100FF000284670BD022070BD022684F82160A063DF
:101000002068066826F0010606602046FFF768FDA6
:10101000E06A00282068016802D041F00E0106E075
:1010200021F0040101602068016841F00A010160BB
:101030002068016841F001010160D9E770B50446FC
:1010400000F004F90546601C02D00448007804440E
:1010500000F0FCF8401BA042FAD370BD0C00002049
:101060002DE9F84FDFF8B8910024A9F1040B2346CD
:101070000F2709F1040AABF1040EC9E00125A540D0
:101080002A40AA427DD1674ED1F804C0ACEB0608D5
:10109000B44532D014DCBCF1030F3AD009DCBCF10A
:1010A000000F2AD0BCF1010F1CD0BCF1020F31D1CE
:1010B0001DE0BCF1110F17D0BCF1120F2AD119E0BD
:1010C000B8F5881F19D006DCB8F5803F15D0B8F503
:1010D000801F1FD111E0B8F5001F0ED0B8F5041F16
:1010E00018D10AE0CB6815E0CB681B1D12E0CB6875
:1010F00008330FE0CB680C330CE08B682BB1012B6D
:101100004FF0080303D0456104E0042302E00561C9
:1011100000E00023FF2A01D8064601E000F10406A2
:101120004FEA840501D9A5F12005D6F8008007FA19
:1011300005FC28EA0C0803FA05F548EA0508C6F894
:1011400000804D68ED0062D5374DAE6946F001066E
:10115000AE61AD6924F0030605F001050095334D3D
:1011600006EB050CDCF80850A607360F07FA06F860
:1011700025EA0805DFF8B880404503D14FF00008A4
:1011800017E044E0DFF8AC80404502D14FF00108A1
:101190000FE0DFF8A480404502D14FF0020808E0DC
:1011A000DFF89880404502D14FF0030801E04FF08E
:1011B000040808FA06F848EA0508CCF808804D68E3
:1011C000D9F80060ED024D4601D5164300E0964384
:1011D0002E604D68DAF80060AD02554601D5164321
:1011E00000E096432E604D68DBF80060AD035D467D
:1011F00001D5164300E096432E604D68DEF800608E
:10120000ED03754601D5164300E096432E60641C3D
:101210000D682A46E5407FF431AFBDE8F88F000045
:1012200008040140000011100010024000000140BD
:1012300000080140000C0140001001400014014072
:101240000AB1016170470904FBE7000001488068AA
:10125000704700000C0000200248816802781144A9
:10126000816070470C000020074810B5016841F00C
:1012700010010160032000F07BF80F2000F006F859
:1012800000F024F8002010BD0020024070B50D4D84
:1012900004464FF47A712878B1FBF0F00A490968E6
:1012A000B1FBF0F000F026FD48B9102C07D2002267
:1012B0002146501E00F03CF800206C6070BD0120FB
:1012C00070BD00000C000020180000200F4808B579
:1012D000816941F001018161816901F001010091A1
:1012E000C16941F08051C161C069002200F08050A5
:1012F00000900F21901E00F01BF80548416821F076
:10130000E06141F00071416008BD00000010024042
:1013100000000140002809DB00F01F02012191407C
:101320004009800000F1E020C0F800117047000083
:10133000F0B40E4B1B680C46C3F30223C3F1070540
:10134000042D00D90425191D072901D2002300E02E
:10135000DB1E012606FA05F1491E214099409E40F8
:10136000761E16403143F0BC01F0E7BC0CED00E006
:10137000064900F0070208684FF6FF03184040EAEC
:101380000220034A10430860704700000CED00E0A3
:101390000000FA052DE9F0470F46050061D0434EE5
:1013A000306800F00700B84209D2306820F007002A
:1013B00038433060306800F00700B84251D12868E7
:1013C0003B4C810712D5400703D5606840F4E060CC
:1013D00060602878000703D5606840F46050606062
:1013E0006068A96820F0F000084360602878C007B2
:1013F00028D06868012810D02168022810D08907F9
:1014000000292EDA616821F0030101436160FFF7D2
:101410001DFF804641F288390DE021688903EFE71E
:101420008901EDE7FFF712FFA0EB0801494502D95A
:101430000320BDE8F0876068696800F00C00B0EB3D
:10144000810FEFD1306800F00700B8420BD9306847
:1014500020F0070038433060306800F00700B842E1
:1014600001D00120E5E72878400705D56068E968E4
:1014700020F4E060084360602878000706D56068C3
:10148000296920F4605040EAC100606000F038F83B
:101490006168084AC1F30311515CC84006490860FD
:1014A00006480068FFF7F2FE0020C2E70020024075
:1014B00000100240F64A000818000020100000202A
:1014C0000448054900684968044AC1F30221515C97
:1014D000C84070471800002000100240064B00086A
:1014E0000448054900684968044AC1F3C221515CB7
:1014F000C84070471800002000100240064B00084A
:101500002DE9F0411D494A681D4802F00C03042BE7
:101510002ED0082B2CD11B48C2F38343C45CD003CC
:1015200028D5C86A174A00F00F000E32105CCA6A4C
:10153000D20316D5CA6AC96AC2F30312C1F30321E2
:10154000521C891CA2FB0023A1FB04150C4F002692
:10155000A1FB070C05FB07C501FB0651FEF710FFB9
:1015600003E007496143B1FBF0F00D2C00D14008C6
:10157000BDE8F08104486043FAE700000010024033
:1015800000127A00D84A000800093D002DE9F84F02
:10159000040070D02078F14DC00749D06868C0F3CE
:1015A0008100012807D06868C0F38100022809D1B2
:1015B0006868C00306D52868800339D5A06800286C
:1015C000E7D035E0A068B0F5803F0BD010B1B0F5A2
:1015D000A02F11D0286820F480302860286820F4DB
:1015E000802002E0286840F480302860A06890B134
:1015F000FFF72CFE06460AE0286840F480202860A9
:10160000F0E700BFFFF722FE801B642876D8286829
:101610008003F7D50CE0FFF719FE064605E000BF92
:10162000FFF714FE801B6428F0D828688003F7D4E5
:101630002078CB4E80074FF001094FF000073AD5D4
:10164000686810F00C0F07D06868C0F381000228AA
:1016500009D16868C00306D42868800715D5606979
:10166000012808D111E06069B8B1C6F80090FFF711
:10167000EDFD804606E042E1FFF7E8FDA0EB080043
:101680000228C3D828688007F6D52868A16920F009
:10169000F80040EAC10028600DE03760FFF7D6FD92
:1016A000804605E0FFF7D2FDA0EB08000228ADD888
:1016B00028688007F6D4207800072ED5A948E1696C
:1016C000E9B1C0F80090FFF7C1FD804606E000BF19
:1016D000FFF7BCFDA0EB0800022897D8686A8007D6
:1016E000F6D5A1484FF4FA510068B0FBF1F0009034
:1016F00000BF0098411E0091FAD20EE0B0E00760F2
:10170000FFF7A4FD804605E0FFF7A0FDA0EB080071
:10171000022889D8686A8007F6D42078400763D504
:10172000E8694FF00008C00009D4E86940F0805033
:10173000E861E8694FF0010800F0805000908B48A4
:101740000168C90512D40168834641F480710160C3
:10175000FFF77CFD824605E0FFF778FDA0EB0A006D
:1017600064287DD8DBF80000C005F5D52069012884
:101770000AD008B1052813D0286A20F00100286299
:10178000286A20F0040002E0286A40F00100286284
:10179000206941F2883B98B1FFF758FD82460BE083
:1017A000286A40F004002862EEE700BFFFF74EFD14
:1017B000A0EB0A01594553D8286A8007F6D50CE0FA
:1017C000FFF744FD824605E0FFF740FDA0EB0A016C
:1017D000594545D8286A8007F6D4B8F1000F03D0E0
:1017E000E86920F08050E861E06AD0B36968C90315
:1017F00007D56968C1F38101022902D1E96AC903E9
:101800007DD4022808D0E86A20F48030E862B76608
:10181000FFF71CFD80463BE02868C00005D5E86A5C
:10182000616B00F0F000884269D1B766FFF70EFDEA
:10183000804605E0FFF70AFDA0EB0800642874D895
:1018400028680001F6D4E86A616B20F0F0000843D4
:10185000E862E86A216B20F470600843E86201E006
:1018600063E018E0C6F86890FFF7F0FC804605E0FA
:10187000FFF7ECFCA0EB0800642856D828680001AC
:10188000F6D508E0FFF7E2FCA0EB080064284CD88E
:1018900028680001F6D4206A90B36968C1F3810119
:1018A000022949D00228376603D0FFF7CFFC04464F
:1018B0003EE0FFF7CBFC074605E000BFFFF7C6FCA4
:1018C000C01B022831D828688001F7D4606AB0F5BF
:1018D000803F09D1E86A61680843E862E86AE16824
:1018E00020F00F000843E862D4E909010843696861
:1018F00021F4741108436860C6F8609001E028E0A4
:1019000029E0FFF7A3FC044605E000BFFFF79EFCBB
:10191000001B022809D828688001F7D51BE000BF0A
:10192000FFF794FC001B022802D90320BDE8F88FC2
:1019300028688001F4D40EE00128F7D06868626A54
:1019400000F48031914204D1A16A00F47010884201
:1019500001D00120EAE70020E8E700000010024083
:101960000000424280044242180000200070004003
:10197000704790F85100704770B5040009D0606A54
:10198000002540B125616561A56294F8510040B120
:101990000CE0012070BD6068B0F5827FF4D0E56195
:1019A000F2E784F85050204600F040F8022084F816
:1019B00051002068016821F040010160A088218960
:1019C00000F4827001F404410843A18901F400612C
:1019D0000843217C01F002010843217D01F001014F
:1019E0000843218B01F400710843217F01F0380185
:1019F000084394F8201001F080010843218D01F480
:101A00000051084321680860A069042101EA1040E0
:101A1000216848602068C16921F40061C161656581
:101A2000012084F85100002070BD000070B586B020
:101A300000250646009501950295039500681A4910
:101A400088422ED11949886940F48050886188699C
:101A500000F480500490886940F00400886188692F
:101A6000694600F004000490A0200090022001903C
:101A7000032003900E48FFF7F3FA0F4C0D48206047
:101A80001020C4E901058020C4E903056561A56152
:101A90002046E561FFF75CFA08B1FFF737F8B46458
:101AA000666206B070BD00000030014000100240C8
:101AB0000008014030000240480100202DE9F84FA5
:101AC000984616468A460446FFF7C0FB814694F8BE
:101AD000510001281ED1BAF1000F73D0002E71D031
:101AE00094F85000012815D0012784F85070032085
:101AF00084F8510000256565C4F830A0A686E68606
:101B0000A563A587E58765642564A068B0F5004FE7
:101B100003D00CE00220BDE8F88F2068016821F0B6
:101B2000400101602068016841F480410160206843
:101B30000168490603D4016841F040010160E06892
:101B4000B0F5006F606803D048B3012E27D047E09E
:101B500008B1012E1FD1206B21680088C86006E003
:101B600020688168890709D5216B0988C160206BCD
:101B7000801C2063E08E401EE0860CE0FFF766FBD1
:101B8000A0EB0901414503D3B8F1FF3F03D035E095
:101B9000B8F1000F32D0E08E0028E1D123E0206BB5
:101BA00021680078087306E02068816889070AD5F3
:101BB000216B09780173206B401C2063E08E401E6E
:101BC000E0860DE02BE0FFF741FBA0EB090141456A
:101BD00003D3B8F1FF3F03D010E0B8F1000F0DD0F0
:101BE000E08E0028E0D14A464146204600F022FE21
:101BF00008B120206065A06830B109E084F8517018
:101C000084F85050032086E72068C16880680090FF
:101C100084F8517004F8505F60680028F3D0012008
:101C200079E7000070B5044690F8510001281CD1F6
:101C3000C9B1C2B194F85000012816D0012084F82F
:101C40005000032084F85100002565652163A286B9
:101C5000E286A56365642564A587E587A068B0F57D
:101C6000004F04D00DE0012070BD022070BD20683F
:101C7000016821F0400101602068016841F4804161
:101C80000160A16C1748C862A16C17488862A16CFA
:101C900016480863A06C4563E38E2268216B0C3202
:101CA000A06CFFF793F930B1606D40F010006065F3
:101CB00084F85050D7E720680168490603D40168CA
:101CC00041F04001016084F850502068416841F0C3
:101CD000200141602068416841F00201416000201C
:101CE00070BD0000C7270008D1270008A5270008FD
:101CF0007047704710B5401EB0F1807F01D30120BE
:101D000010BD4FF0E02460610F21601701F015F85D
:101D10000020A06107202061002010BD70B590F860
:101D20003C20012A29D0012480F83C40022280F87E
:101D30003D2003685A689D6822F070060A683243A5
:101D40005A600F4B02689A420BD0B2F1804F08D014
:101D50000C4B9A4205D00C4B9A4202D00B4B9A4244
:101D600004D1496825F080031943916080F83D4013
:101D7000002180F83C10084670BD022070BD0000B4
:101D8000002C01400004004000080040000C00400E
:101D900000B585B000210091019102910391006886
:101DA000104988421BD11048816941F010018161BE
:101DB0008069694600F0100004904FF47070009044
:101DC0000220019003900948FFF74AF9084841684A
:101DD00021F4406141F0E06141F44061416005B0AF
:101DE00000BD00000004004000100240001001404F
:101DF0000000014070B5044690F83C0000260D46F6
:101E000001280FD0012084F83C006AB1042A1DD0BB
:101E1000082A2FD00C2A3FD00126002084F83C004D
:101E2000304670BD022070BD206800F015FE2068AD
:101E3000816941F0080181612068816921F0040114
:101E40008161206881692A69114311E0206800F0EE
:101E50002BFE2068816941F40061816120688169FD
:101E600021F480618161206881692A6941EA022147
:101E70008161D2E7206800F043FE2068C16941F02B
:101E80000801C1612068C16921F00401C1612068B5
:101E9000C1692A69114311E0206800F05DFE2068E5
:101EA000C16941F40061C1612068C16921F48061A8
:101EB000C1612068C1692A6941EA0221C161ACE7B8
:101EC00010B5040003D094F83D0010B107E00120E4
:101ED00010BD002084F83C00204600F01FF80220CE
:101EE00084F83D00211D206800F064FD012084F885
:101EF000460084F83E0084F83F0084F8400084F8EF
:101F0000410084F8420084F8430084F8440084F8D7
:101F1000450084F83D00002010BD000008B50068B1
:101F20000649884208D10648C16941F00201C161F1
:101F3000C06900F00200009008BD000000040040ED
:101F40000010024010B50446022249B104290ED007
:101F5000082913D094F84100012816D0012010BDA3
:101F600094F83E000128F9D184F83E200FE094F85F
:101F70003F000128F2D184F83F2008E094F84000A7
:101F80000128EBD184F8402001E084F841200122AF
:101F9000206800F053FD11492068884203D1426C4B
:101FA00042F400424264206888420BD0B0F1804F76
:101FB00008D00B49884205D00A49884202D00A4914
:101FC000884204D1816801F00701062903D0016825
:101FD00041F001010160002010BD0000002C014013
:101FE0000004004000080040000C004030B50446EA
:101FF0000D460068002200F021FD174B41F211113F
:1020000020688A10984209D1036A0B4206D1036AFC
:10201000134203D1436C23F4004343642068036AF2
:102020000B4206D1016A114203D1016821F001017E
:10203000016001203DB1042D08D0082D09D084F89D
:102040004100002030BD84F83E00FAE784F83F00EC
:10205000F7E784F84000F4E7002C014070B5040075
:1020600004D094F84100002510B106E0012070BDB5
:1020700084F84050204600F023F8242084F84100E2
:102080002068C16821F40051C160204600F0F8FDCD
:102090002068016921F4904101612068416921F0C3
:1020A0002A0141612068C16841F40051C160656442
:1020B000202084F8410084F842006563002070BD50
:1020C00030B585B000240094019402940394006814
:1020D000194988422DD11948C16941F48021C16153
:1020E000C16901F480210491816941F0100181618D
:1020F0008069134D00F0100004904FF48060009050
:10210000022001900320039069462846FEF7A8FFAD
:10211000E814CDE90004694628460294FEF7A0FFC2
:102120000848416821F0300141F0E06141F01001C0
:10213000416005B030BD0000004800400010024082
:102140000010014000000140FEE72DE9F041070AC0
:10215000C6B20021F0238722084600F009F94FF6A5
:1021600020500446FEF7B6F805000FD000202918CD
:102170002F54801C4E70A042F9D32146284600F00F
:1021800091F92846BDE8F041FEF7D3B8BDE8F081EB
:102190002DE9FF5F8A468146134902EB420001EBBD
:1021A0008000A0F5C07800254FF0010B00240BFA49
:1021B00005F6AAEB050700BF18F80400B9B23042D3
:1021C00009EB040080B201D0039A00E00E9A00F0FF
:1021D0000DF8641CE4B20C2CEED36D1CEDB2062D90
:1021E000E4D3BDE8FF9F0000584B000838B5144603
:1021F00001231A4600F0BCF8200A8DF800008DF883
:1022000001400221684600F025F938BD2DE9F84368
:102210008046C1F1EF001F46154684B2089E08E0D3
:102220003B46214640460096FFF7B2FFA41FA4B2EA
:102230006D1C2A78002AF3D1BDE8F88310B5414C13
:102240008AB0002210212046FEF7FAFF3220FEF766
:10225000F5FE012210212046FEF7F2FF3220FEF7A4
:10226000EDFE362000F0B6F8602000F0D3F83A20FA
:1022700000F0B0F8052000F0CDF8B22000F0AAF888
:1022800031A1D1E90001CDE90801052108A800F03C
:10229000E1F8B72000F09EF8352000F0BBF8BB2035
:1022A00000F098F8192000F0B5F8C02000F092F87E
:1022B0002C2000F0AFF8C22000F08CF8012000F0D4
:1022C000A9F8C32000F086F8122000F0A3F8C4207B
:1022D00000F080F8202000F09DF8C62000F07AF889
:1022E0000F2000F097F8D02000F074F8A42000F040
:1022F00091F8A12000F08EF8E02000F06BF814A017
:102300000FC88DE80F000E21684600F0A3F8E12009
:1023100000F060F812A104AC0FC984E80F000E2190
:1023200004A800F097F8212000F054F8112000F0E4
:1023300051F87820FEF782FE292000F04BF80AB011
:1023400010BD0000001001400C0C003333000000F1
:10235000D0040D11132B3F544C180D0B1F230000FC
:10236000D0040C11132C3F44512F1F1F20230000B9
:102370002DE9FC4100F1340401F12807A518FE18ED
:102380002A206D1E761E00F025F8200A8DF8000028
:102390008DF80140280A8DF802008DF803500421C1
:1023A000684600F057F82B2000F014F8380A8DF832
:1023B00004008DF80570300A8DF806008DF807606E
:1023C000042101A800F046F82C2000F003F8BDE835
:1023D000FC81000031B5002220210B48FEF730FFC0
:1023E0000A4C002210212046FEF72AFF4FF0FF334F
:1023F000012269460648FFF761FB012210212046B1
:10240000FEF71EFF38BD000000100140000801402B
:10241000F000002031B5012220210B48FEF710FF0B
:102420000A4C002210212046FEF70AFF4FF0FF332E
:10243000012269460648FFF741FB01221021204690
:10244000FEF7FEFE38BD000000100140000801400C
:10245000F000002070B50C460546402903D9BDE8C0
:10246000704000F01FB8012220210B48FEF7E8FE63
:102470000A4E002210213046FEF7E2FE4FF0FF33F5
:10248000224629460648FFF719FB3046BDE8704052
:1024900001221021FEF7D4BE0010014000080140C7
:1024A000F000002070B50C460546012220210D48A1
:1024B000FEF7C6FE0C4E002210213046FEF7C0FE8D
:1024C000224629460948FFF7ADFB0848FFF751FAB5
:1024D0000128FAD13046BDE8704001221021FEF7F4
:1024E000AFBE00000010014000080140F0000020D5
:1024F0000D4810B50B490160102141600021816039
:10250000C16001614161017641768176C1760177D2
:102510004177FEF7FDFA002803D0BDE81040FEF732
:10252000F5BA10BD00640040A00000200D4810B5B1
:102530000B4901601021416000218160C16001618F
:102540004161017641768176C17601774177FEF768
:10255000DFFA002803D0BDE81040FEF7D7BA10BD5F
:1025600000680040C8000020094808B5416941F0F2
:10257000010141614069002200F001000090052145
:102580000D20FEF7D5FEBDE808400D20FEF7C2BEC7
:102590000010024010B5074A0021074800F0B6FCC1
:1025A000064C074A00216060064800F0AFFC20603E
:1025B00010BD0000B44A00082129000800000020D6
:1025C000104B00089D2B00082DE9F04186B0002437
:1025D00028480094019402940394816941F02001F9
:1025E0008161816901F020010491816941F0040158
:1025F0008161816901F004010491816941F0100158
:102600008161816901F010010491816941F0080143
:1026100081618069DFF8608000F00800049000228A
:1026200050214046FEF70CFE144F00223021384660
:10263000FEF706FE502001250226CDE90005CDE972
:10264000024669464046FEF70BFD3020CDE9000505
:10265000CDE9024669463846FEF702FD4FF4407068
:10266000CDE90004694640460294FEF7F9FC06B045
:10267000BDE8F08100100240000801400010014058
:10268000104810B50E4901604FF48271416000217D
:102690008160C1604FF400720161C0E90512082237
:1026A000C0E90721416281620A21C162FFF764F932
:1026B000002803D0BDE81040FEF728BA10BD000086
:1026C00000300140F000002010B58AB000240794CB
:1026D0001C2168460894FDF7C4FF22482049C0E940
:1026E00000144FF6FF71C0E9024104618461FFF7F5
:1026F000E7FB08B1FEF70AFA079407A919480894FE
:10270000FFF70CFB08B1FEF701FA6020CDE90004E9
:1027100002940022694613480494FFF76BFB08B14A
:10272000FEF7F4F9042269460E48FFF763FB08B18F
:10273000FEF7ECF9082269460A48FFF75BFB08B18F
:10274000FEF7E4F90C2269460648FFF753FB08B18F
:10275000FEF7DCF90348FFF71BFB0AB010BD0000D1
:10276000000400408C0100200C4810B50A490160AB
:102770004FF4E1314160002181600C22C160C0E969
:1027800004128161C161FFF769FC002803D0BDE834
:102790001040FEF7BBB910BD00480040D401002036
:1027A000FEE7FEE710B5406A01684A6822F00302BE
:1027B0004A60416D41F010014165012180F85110DE
:1027C000FFF7D6F810BD10B5406AFFF792FA10BDBA
:1027D00038B50546446AFEF739FD024628680068A8
:1027E000800623D42068416821F0200141602068E0
:1027F000416821F0020141606421204600F01AF88E
:1028000018B1606D40F020006065A068002118B923
:102810002068C26880680090E186012084F8510039
:10282000606D18B12046FFF7A3F838BD2046FFF7CA
:102830005FFA38BDF8B515460E460B4600920446C1
:102840000122022100F010F840B933460022802115
:102850002046009500F008F8002804D0606D40F094
:10286000200060650320F8BD2DE9F8431E4691461F
:1028700088460446089DFEF7E9FC401B351AFEF722
:10288000E5FC074625480068C0F3CB30684338E0D4
:10289000701C37D0FEF7DAFCC01BA84203D215B17A
:1028A000009860B32CE02068416821F0E0014160AD
:1028B0006068B0F5827F0BD1A068B0F5004F02D000
:1028C000B0F5806F04D12068016821F040010160FB
:1028D000A06AB0F5005F09D12068016821F40051B9
:1028E00001602068016841F400510160012084F812
:1028F0005100002084F850000320BDE8F883002533
:10290000401E00902068816838EA010004D0002150
:102910004945BDD10020F0E70121F9E7180000206A
:1029200010B500F0F0FABDE8104000F034BB10B56F
:10293000FEF792FC01F03CFD012803D0BDE81040F9
:1029400001F064BA10BD000070B594B0382168463B
:10295000FDF787FE14210EA8FDF783FE0125002454
:102960002804CDE902040226CDE90860009505950A
:1029700001944FF4E010CDE90A046846FEF706FE24
:1029800008B172B6FEE70F20CDE90E064FF4806065
:10299000CDE9104002210EA81294FEF7FBFC08B10D
:1029A00072B6FEE70148056714B070BD00004242F0
:1029B00070470000F0B502681C4B1D4C1D4D1E4EAB
:1029C0004FF08047984207D0B84205D0A04203D0CC
:1029D000A84201D0B04204D122F0700C4A6842EA09
:1029E0000C02984207D0B84205D0A04203D0A842BA
:1029F00001D0B04203D122F44074CA6822434C692A
:102A000022F08002224302608A68C2620A688262FF
:102A1000984201D109690163012141610169C90736
:102A200003D0016921F001010161F0BD002C0140DA
:102A30000004004000080040000C004010B501F008
:102A40001F030121046A99408C430462016A9A4081
:102A50001143016210BD000030B5036A026A22F022
:102A6000010202624268846924F073050C682C43F9
:102A700023F002058B682B430A4DA8420BD123F0AB
:102A80000805CB6822F440722B434D6923F0040300
:102A900015438A692A43426084614968416303623D
:102AA00030BD0000002C014030B5026A036A23F0FB
:102AB00010030362436884690D6824F4E64444EA21
:102AC00005248D6822F0200242EA05120B4DA8422F
:102AD0000ED1CD6822F0800242EA05124D6923F43E
:102AE000406343EA85038D6922F0400243EA85038F
:102AF0004360846149688163026230BD002C0140FB
:102B000030B5036A026A22F4807202624268C469C4
:102B100023F4007324F073050C682C438D6843EA9A
:102B200005230C4DA8420ED1CD6823F4006343EA7F
:102B300005234D6922F4405242EA05128D6923F4BF
:102B4000806342EA05124260C4614968C16303625E
:102B500030BD0000002C014030B5046A026A22F446
:102B6000805202624268C3690D6823F4E64343EA77
:102B700005238D6824F4005444EA0534064DA84228
:102B800004D14D6922F4804242EA85124260C36159
:102B900049680164046230BD002C014010B500F0AA
:102BA00063F9074A0021074800F0B0F906490860B8
:102BB00000F08CF900F0A7F9BDE8104000F0EBB987
:102BC000344B0008CD2B0008F01E002086B000F02A
:102BD00036F9064600F02CF90446FFF72FFB0020DB
:102BE000FFF7B3FA4FF47840FFF7AFFA00274FF63C
:102BF000FF752B4616A2394638460097FFF706FBAD
:102C0000002315A2194632200095FFF7FFFA002293
:102C100011461046FDF716FF002211460220FDF76F
:102C200011FF3444224613A101A8FDF721FC2B46D5
:102C300001AA142100200097FFF7E8FA00220221E0
:102C40000120FDF7FFFE204600F0DBF8E9E7000079
:102C500048656C6C6F0000007468697320697320AC
:102C60007369636B2028445433352D64726976652B
:102C7000722900005469636B3A20256C75000000CE
:102C800070B5044600680169E26821F440511143BF
:102C900001612169A0680843616908432168CA6825
:102CA00041F20C639A430243CA6020684169A269F9
:102CB00021F44071114341611E492068884202D1CC
:102CC000FEF70EFC01E0FEF7FBFB00EBC00101EBA1
:102CD0000012606864218000B2FBF0F3B3FBF1F3F3
:102CE0006FF018067343B2FBF0F5B2FBF0F605EB9C
:102CF0008305322303EB0515B5FBF1F5B6FBF1F6C1
:102D000005F0F00505EB0615B2FBF0F6B2FBF0F0AE
:102D1000B0FBF1F06FF01802504306EB800003EBBC
:102D20000010B0FBF1F0216800F00F00284488602B
:102D300070BD000000380140FEE70907090E0028B9
:102D400004DB00F1E02080F80014704700F00F0071
:102D500000F1E02080F8141D704700002DE9F041DB
:102D6000040006D0184E306884420AD10020BDE825
:102D7000F081502080F31188BFF34F8FBFF36F8F26
:102D8000FEE700F0C9FD6569776BB66B00F0E4FD06
:102D9000BD4201D0B54201D10220E8E70B4885428F
:102DA00008D1A06A0028F7D194F858000128F3D080
:102DB0000320DCE705481438854202D00DB101201C
:102DC000D5E70420D3E700001C0000200C070020FA
:102DD000FEF74AFAFFF7B8FDFFF7F6FBFFF7C4FB73
:102DE000FFF74EFCFFF770FCFFF782FBFFF79EFB3F
:102DF000FFF7BAFC00F026F8FFF7CCFB00F04AF82A
:102E0000FEE738B50546EFF3058010B16FF0050415
:102E10000CE0002401F0DAFA291A0090002903DD01
:102E2000684600F051FE01E06FF00304204638BD13
:102E3000EFF3058008B101F0CFBA01F0C7BA4FF443
:102E40007A707047EFF3058010B16FF0050070479E
:102E50000448016811B14FF0FF3070470121016053
:102E6000002070476C00002010B5EFF3058010B112
:102E70006FF0050010BD01F09BFA20B1022804D0CC
:102E80004FF0FF3010BD012010BD00F031FF0020D9
:102E900010BD000010B5EFF3058010B16FF0050014
:102EA00010BD08480168012902D04FF0FF3010BD65
:102EB000054A002182F8141D0221016000F0D4FEB1
:102EC000002010BD6C0000200BE000E070B5EFF3B7
:102ED000058010B16FF0050413E001F069FA4FF0BE
:102EE000FF3510B102280BD108E0012401F058FB96
:102EF000012806D001F05CFA10B102E0002400E0E5
:102F00002C46204670BD01F04DBA00002DE9FF416E
:102F10004FEA01034FF00005EFF30581039549BB2C
:102F200040B38027182100244AB3166806B13446FE
:102F300096691EB13146761E382E02D21679F607F2
:102F400003D0002004B0BDE8F081566906B1B7088F
:102F5000D2F808C0BCF1000F0DD0D5685C2D18D395
:102F600012693AB136B18DE806103A46214601F0B1
:102F7000EEF903900DE0D6685EB912694AB903AA6A
:102F8000CDE90012BAB2214601F0B4F9012800D00F
:102F900003950398D6E770B50546EFF3058010B1A9
:102FA0006FF005040FE04DB12846FFF7D7FE042867
:102FB00007D00024284600F0CDFD04E06FF00304A4
:102FC00001E06FF00204204670BD00002DE9F041E1
:102FD000134C0F460546E6682068001D00F040FCD3
:102FE000681C07D137B12168BDE8F0410D48091DC3
:102FF00000F086BC20683544B5424560216805D2A2
:10300000A06BBDE8F041091D00F062BC606B091DBA
:1030100000F05EFCA06A854200D2A562BDE8F081A6
:103020001C0000200C0700202DE9F041054600F0AF
:1030300073FC2D4CA068401CA06020682B4F10B181
:10304000606930B32BE02560A068012827D10026F5
:1030500006EB860007EB800000F02CFC761C382E77
:10306000F6D3234800F026FC2148143000F022FC5F
:103070001F48283000F01EFC1D483C3000F01AFCB0
:103080001B48503000F016FC194860631430A063F0
:1030900005E02068E96AC06A884200D82560606A55
:1030A000401C60626864E86A2169884200D9206136
:1030B00000EB800007EB8000291D00F021FC00F0F0
:1030C0004BFC606900280CD02068E96AC06A88421D
:1030D00007D208494FF080500860BFF34F8FBFF30D
:1030E0006F8FBDE8F08100001C0000205C02002012
:1030F000BC06002004ED00E038B500F00DFC104CDB
:103100002068C8B90F4800F0D5FB0E48143000F015
:10311000D1FB0C48E060143020610A4B0020F03BEA
:10312000009003F1500210210A2000F085FE20607B
:1031300010B105A100F092FCBDE8384000F00CBCD5
:103140005800002010080020546D7251000000004B
:1031500030B4026C0B46002A0BD0C1681144C16028
:103160008468A14201D30168C16030BC1846FDF7F4
:103170002BBA30BC70472DE9F041856B17460446E9
:103180000026026C82B1C7B1E068FDF71DFAE16864
:10319000206C091AE1602268914202D2A168081AE3
:1031A000E060022F16D017E02068A8B9A06801F0EF
:1031B0007FF906460020A0600EE06068FDF704FA83
:1031C000216C606808446060A168884204D320686C
:1031D000606001E005B16D1E6D1CA5633046BDE861
:1031E000F08110B5044690F8590058B101280CD070
:1031F00002280FD0502080F31188BFF34F8FBFF308
:103200006F8FFEE7206B00F0BBFB2046BDE810404F
:1032100000F0B6BB10BD000010484FF480514207CB
:1032200006D0C01D0D4920F00700411AC1F580519C
:103230000B4A00230144C2E900030839183A21F07F
:10324000070111604B600B600B1AC0E9001393601B
:103250004FF000405360506170470000F00E0020B6
:1032600088000020144E154CA6F29C474FF0805861
:10327000DFF84C9012E000BF00F04EFBF068C5682C
:10328000281D00F0EDFAA068401EA0606068401E96
:10329000606000F061FB2846FFF7A3FF606800282C
:1032A000EAD138680128F9D9C9F80080BFF34F8FF7
:1032B000BFF36F8FF2E70000F80600201C0000202B
:1032C00004ED00E070B51D46049C51B1C4F8002027
:1032D000C4E90F010121204600F0E2FD84F84C50C2
:1032E00070BD2460F4E700002DE9F05F8846DDE959
:1032F0000B941546834691009A460A9EA522206BA0
:10330000FDF7A7F96FF00301206B01EB850108447D
:1033100020F00707780707D0502080F31188BFF30B
:103320004F8FBFF36F8FFEE70025B8F1000F0FD06E
:103330005FF00000221818F8001082F8341018F816
:10334000001011B1401C1028F4D384F8435001E060
:1033500084F83450382E00D33726E662C4E913656A
:10336000201D00F0B2FA04F1180000F0AEFA24615A
:10337000C6F138006462A061656584F85850524611
:103380005946384600F05AFA2060B9F1000F01D0D2
:10339000C9F80040BDE8F09F30B5114900E0114682
:1033A0000A688242FBD34B685C18844203D14068B0
:1033B00018444860084643681C18944209D1084CD8
:1033C000183C2468A24209D052681A4442600A6834
:1033D00012680260814200D0086030BD0460F9E7E5
:1033E0008800002070B5002441600B4D00619142BF
:1033F00006D8D11A8269914206D2011D286907E0D8
:103400009A4203D2994201D3012403E0011DE868E6
:1034100000F05EFA204670BD5800002010B504464A
:1034200000F07AFAA06B28B15FF0000400F094FA83
:10343000204610BD0124F9E730B589B03C4D6EE05F
:103440000498002806DADDE90601059A90470498F9
:10345000002864DB069C606910B1201D00F000FAB2
:1034600003A800F0D7F8024604980A2857D2DFE8EC
:1034700000F00505052D334A05052D3394F8280085
:1034800040F0010084F828000599A069059B0144DB
:103490002046FFF7A7FF68B3216A2046884794F8C3
:1034A000280040073BD5002000900598A169002323
:1034B00042181946204601F005F9D8B9502080F38A
:1034C0001188BFF34F8FBFF36F8FFEE714F8280FFB
:1034D00020F00100207022E094F8280040F0010064
:1034E00084F828000598A06128B181181346204669
:1034F000FFF778FF13E0502080F31188BFF34F8F60
:10350000BFF36F8FFEE794F82800810703D42046AD
:1035100000F036FA03E020F0010084F828000022D1
:1035200004A9286800F010FE002889D109B030BD38
:10353000580000202DE9FC410F46054600F0D8FB5D
:1035400001A800F067F80446019818B101F028F8C6
:10355000BDE8FC81254EAFB130690068D0B30027CB
:10356000291B3A46306800F08DFA01F019F800285E
:10357000EED11F494FF080500860BFF34F8FBFF36B
:103580006F8FE5E7A542EBD801F00AF8F06827460F
:10359000C068C468201D00F063F994F82800410752
:1035A00019D5A0692B4641193A462046FFF71AFF64
:1035B000A8B100200346014600902A46204601F0AB
:1035C00081F860B9502080F31188BFF34F8FBFF3AB
:1035D0006F8FFEE707E020F0010084F82800216AE1
:1035E00020468847B4E70127BAE7000058000020CA
:1035F00004ED00E00648416B096829B1416BC968D8
:10360000C9684968816270474FF0FF31FAE70000EE
:103610001C00002070B5054600F0D8FE064E04469A
:10362000B068844203D200F009F8012000E00020D5
:1036300028602046B46070BD58000020F8B5194DD0
:1036400020E0C068C4680668201D00F009F9216AFE
:103650002046884794F82800400713D5A0693044D5
:10366000B04206D924616060211DE86800F030F99D
:1036700008E000200346014600903246204601F053
:1036800021F838B1E86801680029DAD12969C5E96B
:103690000310F8BD502080F31188BFF34F8FBFF3A4
:1036A0006F8FFEE75800002008484068401C4FF02C
:1036B000500080F3118804D0BFF34F8FBFF36F8F9A
:1036C000FEE7BFF34F8FBFF36F8FFEE79000002040
:1036D000074CE068016841B1C0680021D0F80000E3
:1036E000FFF728FFFFF7A8FEF3E701210020F7E727
:1036F000580000202DE9F041044600F00DF994F93E
:10370000455004F1240609E0606A48B1304600F0F3
:103710000FFF08B100F06EFA6D1E6DB2002DF3DCE4
:103720004FF0FF3684F8456000F016F900F0F4F829
:1037300094F9445004F1100709E0206948B1384673
:1037400000F0F6FE08B100F055FA6D1E6DB2002DC6
:10375000F3DC84F84460BDE8F04100F0FDB80000FF
:103760002DE9F0410546002700F0C2FA324E3068DC
:1037700008B9FFF751FD706905424ED1C5B3083550
:1037800068070ED005F00700C0F10800054468077F
:1037900007D0502080F31188BFF34F8FBFF36F8F96
:1037A000FEE72DB37068854237D8234818300146AC
:1037B0000C6801E020460C466168A94202D22168EB
:1037C0000029F7D131688C4227D007682168016051
:1037D00060680837411B10290FD96019420708D0CB
:1037E000502080F31188BFF34F8FBFF36F8FFEE738
:1037F00013E041606560FFF7CFFD61687068401AB3
:103800007060B268904200D2B060706901430020DD
:10381000C4E90001F068401CF06000F0C1FE7807C8
:1038200007D0502080F31188BFF34F8FBFF36F8F05
:10383000FEE73846BDE8F0817000002010B5031F98
:103840004FF080741C601B1F21F001011960191FCB
:10385000024B0B60143940380A6010BDA9360008CD
:10386000D0E9013201699A60D0E901235A604A68BF
:10387000824201D182684A60002202610868401ECB
:103880000860086870470000034B036003F15C00A8
:10389000086080201060704738080020044B0360E7
:1038A00003F15C0008604FF4807010607047000006
:1038B000940A002000F108014FF0FF32C0E9011224
:1038C000C160016100210160704700210161704702
:1038D00030B50B685A1C02D000F1080202E0026900
:1038E00004E02246546825689D42FAD953684B602B
:1038F00099608A60516008610168491C016030BDAF
:1039000042684A6093688B6093685960916008616F
:103910000168491C01607047502080F31188BFF393
:103920004F8FBFF36F8F0A494868401C48600128D9
:103930000CD10848006810F0FF0F07D0502080F32A
:103940001188BFF34F8FBFF36F8FFEE77047000002
:103950009000002004ED00E00849486828B1401EAE
:10396000486001D180F311887047502080F311889E
:10397000BFF34F8FBFF36F8FFEE700009000002072
:1039800070B500282AD0164DA0F108046068696956
:10399000084207D1502080F31188BFF34F8FBFF347
:1039A0006F8FFEE722683AB1502080F31188BFF391
:1039B0004F8FBFF36F8FFEE78843606000F098F988
:1039C00060686968084468602046FFF7E5FC28697C
:1039D000401C2861BDE8704000F0E2BD70BD0000F1
:1039E000700000204FF0E020002101618161054955
:1039F0004FF47A720968B1FBF2F1491E4161072167
:103A0000016170471800002010B5FCF73FFC114918
:103A100010280ED300F1E02090F8F0030A789042CD
:103A200007D2502080F31188BFF34F8FBFF36F8F01
:103A3000FEE709480068896800F4E060884207D919
:103A4000502080F31188BFF34F8FBFF36F8FFEE7D5
:103A500010BD0000900000200CED00E010B5084BF8
:103A6000002200BF53F832401CB1521C082AF9D37F
:103A700010BD43F8321003EBC201486010BD0000D6
:103A80001C02002070B515460E460446FFF744FFA1
:103A900094F944100020491C01D184F8440094F9A1
:103AA0004510491C01D184F84500FFF755FFA06B74
:103AB00028B92A46314604F1240000F0B9F820461E
:103AC000BDE87040FFF716BE70B50D4604000BD080
:103AD00095B11E4A106BB8B1502080F31188BFF326
:103AE0004F8FBFF36F8FFEE7502080F31188BFF335
:103AF0004F8FBFF36F8FFEE7502080F31188BFF325
:103B00004F8FBFF36F8FFEE700F0F2F8D2682368A3
:103B10005919934204D98B420AD9914202D807E03D
:103B20008B42FAD9881A21600021FFF74FFA00E092
:103B3000216000F035FD002807D105494FF0805085
:103B40000860BFF34F8FBFF36F8F70BD1C00002064
:103B500004ED00E070B50546FFF7DEFE1E4C05B92A
:103B60002568281DFFF77CFEA86A18B105F118002A
:103B7000FFF776FE606A401C60622068854207D1CC
:103B8000291D1648FFF7BCFE6068401C606007E016
:103B9000A068401EA0602846FFF723FBFFF72AFD20
:103BA000FFF7DAFE6069002814D02068854211D141
:103BB000206B38B1502080F31188BFF34F8FBFF3D3
:103BC0006F8FFEE706494FF080500860BFF34F8FBC
:103BD000BFF36F8F70BD00001C000020F8060020AE
:103BE00004ED00E002490A6A0260C968416070475A
:103BF0001C00002001490120C86170471C00002002
:103C000010B50C4650B1094909681831FFF760FE3C
:103C10002046BDE810400121FFF7D8B9502080F3BD
:103C20001188BFF34F8FBFF36F8FFEE71C0000209A
:103C300070B514460D4668B10A4909681831FFF796
:103C40005FFE0CB14FF0FF3521462846BDE87040BD
:103C5000FFF7BCB9502080F31188BFF34F8FBFF33B
:103C60006F8FFEE71C00002030B587B0002403945E
:103C700005AA04A903A80494FFF706FEDDE90301E1
:103C80000094CDE90110002315A11748059A00F012
:103C90005EFB164D0028E8621FD000F0E3FC01280F
:103CA00009D0401C19D1502080F31188BFF34F8FE9
:103CB000BFF36F8FFEE7502080F31188BFF34F8F63
:103CC000BFF36F8F4FF0FF30A86201206861EC6096
:103CD00007B0BDE8304000F045B807B030BD000087
:103CE00049444C4500000000653200081C000020DB
:103CF0000248016B491C0163704700001C00002052
:103D0000164810B5016B11B10121C16110BD002130
:103D1000C1610169124A01E0B9B1491E01EB810399
:103D200052F82330002BF7D001EB810302EB830222
:103D300002F1080453685B685360A34201D15B68D9
:103D40005360DA680260016110BD502080F3118871
:103D5000BFF34F8FBFF36F8FFEE700001C00002002
:103D60005C0200201CB5264908780190FF200870ED
:103D700008788DF800009DF800009DF8002000F004
:103D8000F000904207D0502080F31188BFF34F8F8E
:103D9000BFF36F8FFEE79DF800001A4C00F0500053
:103DA00020700720A06005E09DF8002052008DF8EB
:103DB0000020401E9DF800201206F5D4A0600328C4
:103DC00007D0502080F31188BFF34F8FBFF36F8F60
:103DD000FEE74FF44070A060019808700A4801683F
:103DE00041F470010160016841F070410160FFF72A
:103DF000F9FD00206060FCF713FA00201CBD0000F4
:103E000000E400E09000002020ED00E010B550201C
:103E100080F31188BFF34F8FBFF36F8F00F0E4FA88
:103E200018B104494FF080500860002080F31188D9
:103E300010BD000004ED00E038B5049D18B153B189
:103E4000CAB181B120E0502080F31188BFF34F8FB9
:103E5000BFF36F8FFEE7502080F31188BFF34F8FC1
:103E6000BFF36F8FFEE7502080F31188BFF34F8FB1
:103E7000BFF36F8FFEE739B1502080F31188BFF395
:103E80004F8FBFF36F8FFEE750241C46012384F849
:103E900046302B460094FFF715FA204638BD000047
:103EA00070B50D46040025D0FFF736FDD4E90F208C
:103EB000216802FB0011A1600021A16321686160FB
:103EC0000A46D4E90F01401E00FB0121E1602146B2
:103ED0004FF0FF3001F8440F487004F110008DB12D
:103EE000FFF7E8FC04F12400FFF7E4FCFFF734FDE2
:103EF000012070BD502080F31188BFF34F8FBFF3B6
:103F00006F8FFEE721690029F0D000F011FB002837
:103F1000ECD004494FF080500860BFF34F8FBFF3DF
:103F20006F8FE3E704ED00E02DE9FF4782B01D4607
:103F30008A464FF00008040003D0BAF1000F08D001
:103F400011E0502080F31188BFF34F8FBFF36F8FC4
:103F5000FEE7206C38B1502080F31188BFF34F8FFB
:103F6000BFF36F8FFEE7022D0AD1E06B012807D067
:103F7000502080F31188BFF34F8FBFF36F8FFEE7A0
:103F800000F016FA3F4F4FF000094FF0805648B945
:103F9000049838B1502080F31188BFF34F8FBFF3DE
:103FA0006F8FFEE7FFF7B8FCA06BE16B884207D389
:103FB000022D05D00498D0B1B8F1000F1AD01EE040
:103FC0002A4651462046FFF7D6F8616A19B104F136
:103FD000240000F0ADFA20B13E60BFF34F8FBFF375
:103FE0006F8FFFF7B9FC012006B0BDE8F087FFF73F
:103FF000B3FC22E06846FFF7F5FD4FF00108FFF73C
:10400000ABFCFFF775FEFFF787FC94F94400401CFA
:1040100001D184F8449094F94500401C01D184F802
:104020004590FFF799FC04A9684600F029F930B1E2
:104030002046FFF75FFB00F0B3FA0020D4E7FFF75C
:104040006BFCA06BE16B884213D1FFF785FC04F198
:1040500010000499FFF7D4FD2046FFF74BFB00F05A
:104060009FFA00289ED13E60BFF34F8FBFF36F8F42
:1040700098E7FFF771FC2046FFF73CFB00F090FA51
:1040800090E7000004ED00E02DE9F0471F46904660
:104090008946040003D0B9F1000F08D011E0502088
:1040A00080F31188BFF34F8FBFF36F8FFEE7206C53
:1040B00038B1502080F31188BFF34F8FBFF36F8F5B
:1040C000FEE7022F0AD1E06B012807D0502080F3D1
:1040D0001188BFF34F8FBFF36F8FFEE7FFF794FC9C
:1040E0005020EFF3118680F31188BFF34F8FBFF399
:1040F0006F8FA06BE16B884206D3022F04D00020A3
:1041000086F31188BDE8F08794F94550A06B3A46D4
:1041100049462046FFF72FF8681C04D06D1C84F830
:1041200045500120ECE7606A0028FAD004F1240031
:1041300000F0FEF90028F4D0B8F1000FF1D0012111
:10414000C8F80010EDE700002DE9F747002683B01E
:104150008A46040003D0BAF1000F08D011E05020C5
:1041600080F31188BFF34F8FBFF36F8FFEE7206C92
:1041700038B1502080F31188BFF34F8FBFF36F8F9A
:10418000FEE700F015F9DFF8F4804FF000094FF07A
:10419000805748B9059838B1502080F31188BFF393
:1041A0004F8FBFF36F8FFEE7FFF7B6FBA56BC5B16F
:1041B00051462046FEF7CCFF6D1EA563206950B125
:1041C00004F1100000F0B4F928B1C8F80070BFF392
:1041D0004F8FBFF36F8FFFF7BFFB012006B0BDE825
:1041E000F087059808B11EB106E0FFF7B5FB27E0A0
:1041F0006846FFF7F7FC0126FFF7AEFBFFF778FDF7
:10420000FFF78AFB94F94400401C01D184F84490E4
:1042100094F94500401C01D184F84590FFF79CFBC0
:1042200005A9684600F02CF8002820460AD0FFF7C0
:1042300061FA00F0B5F92046FFF7F0F80028B3D096
:104240000020CBE7FFF7EAF890B104F124000599CC
:10425000FFF7D6FC2046FFF74DFA00F0A1F9002841
:10426000A2D1C8F80070BFF34F8FBFF36F8F9BE7E9
:104270002046FFF73FFA00F093F995E704ED00E0E0
:104280002DE9F0410C46050011D0C4B1FFF744FB05
:10429000174BDA686E682068911B471C17D02F688F
:1042A0001B6A9F4219D0964217D8012410E0502073
:1042B00080F31188BFF34F8FBFF36F8FFEE750205D
:1042C00080F31188BFF34F8FBFF36F8FFEE7002499
:1042D000FFF742FB2046BDE8F081884205D9401A2D
:1042E00020602846FFF77EFCF1E700202060DCE735
:1042F0001C0000202DE9FF5F8346DDE90E8799460B
:1043000016468A469000FFF72BFA05001CD05C2069
:10431000FFF726FA040014D00020256384F8590022
:10432000CDE90240CDE900874B463246514658461A
:10433000FEF7DAFF2046FEF777FE012004B0BDE865
:10434000F09F2846FFF71CFB4FF0FF30F6E7F0B573
:1043500085B0DDE90B640A9DA6B1DCB15C2700974E
:104360002663022684F85960002604AFCDE9024690
:10437000CDE90057FEF7B8FF2046FEF755FE04983A
:1043800005B0F0BD502080F31188BFF34F8FBFF30D
:104390006F8FFEE7502080F31188BFF34F8FBFF37C
:1043A0006F8FFEE701480068704700001C00002086
:1043B0000548416919B1006B18B100207047012010
:1043C00070470220704700001C0000200148C068B0
:1043D000704700001C00002010B5FFF715FB0148D6
:1043E000C06810BD1C0000202DE9F0412E4C0027B4
:1043F000206B28B1A069401CA0613846BDE8F0815F
:10440000E668761CE66013D1606B006838B1502016
:1044100080F31188BFF34F8FBFF36F8FFEE7606BA0
:10442000A16B6163A063206A401C2062FFF7E2F881
:10443000A06ADFF87880864209D3606B0068A0B17B
:10444000606BC068C5686868864211D2A062206847
:10445000C06A00EB800158F82100012800D901272B
:10446000E0690028C9D00127C7E74FF0FF30EDE72A
:10447000281DFFF7F5F9A86A18B105F11800FFF734
:10448000EFF9E86A2169884200D9206100EB8001D8
:1044900008EB8100291DFFF733FAE86A2168C96A31
:1044A0008842CAD30127C8E71C0000205C02002014
:1044B00070B504004FF0000133D01B4D28688442D2
:1044C00007D0502080F31188BFF34F8FBFF36F8F59
:1044D000FEE7206D38B1401E2065E36CE26A9A4227
:1044E0001FD040B11DE0502080F31188BFF34F8FE3
:1044F000BFF36F8FFEE7201DFFF7B2F9E06CE062BB
:10450000C0F13800A061E06A2969884200D92861B9
:10451000064900EB800001EB8000211DFFF7F0F958
:104520000121084670BD00001C0000205C02002034
:1045300070B5C068C46854B104F118000646FFF7AE
:104540008FF9144D286B50B13146134815E05020B7
:1045500080F31188BFF34F8FBFF36F8FFEE7201DED
:10456000FFF77EF9E06A2969884200D928610B4982
:1045700000EB800001EB8000211DFFF7C1F9E06A2C
:104580002968C96A884202D90120E86170BD00200B
:1045900070BD00001C000020E40600205C0200202A
:1045A0002DE9F0472C4D00242746286B38B1FFF742
:1045B000B3F9286B401E2863286B40B146E05020B9
:1045C00080F31188BFF34F8FBFF36F8FFEE7A968A9
:1045D000224E0120D1B3A6F5916980463068E0B142
:1045E000F068C46804F11800FFF73AF9201DFFF7DE
:1045F00037F9E06A2969884200D9286100EB800117
:1046000009EB8100211DFFF77BF9E06A2968C96A7F
:104610008842E3D3C5F81C80E0E70CB1FEF7EAFF5F
:10462000AC694CB14FEA0806FFF7DEFE00B1EE615F
:10463000641EF9D10020A861E86938B10849012752
:1046400038070860BFF34F8FBFF36F8FFFF784F910
:104650003846BDE8F08700001C000020E40600207A
:1046600004ED00E010B586B0FEF746FD114C206861
:10467000B8B100200390049005AA04A903A8FFF78D
:104680000DF9DDE9032102208DE8070000230AA1CE
:104690000B48059AFFF75BFE606010B106B0012081
:1046A00010BD502080F31188BFF34F8FBFF36F8F81
:1046B000FEE7000058000020546D7220537663001E
:1046C000D13600082DE9FF411E46134602000A9D1F
:1046D0004FF0000016D0144C2768002F0FD0CDE902
:1046E00000130292062917DAFFF762FE02284FF044
:1046F00000030FD0002269462068FFF715FC04B0C4
:10470000BDE8F081502080F31188BFF34F8FBFF3D5
:104710006F8FFEE72A46EEE70023324669463846A9
:10472000FFF7B2FCEBE700005800002090EA010F11
:1047300048BF81F0004100F14E81421A3CBF801A0F
:1047400089184FEAD0524FF07F4C1CEA410FA2EB80
:10475000D15318BF9CEA026F00F03B804FF0004C31
:104760004CEA00204CEA012121FA03FC10EB0C0C6E
:104770001ED202F1FF325FEA1C2040EBC25038BF6C
:1047800070471CF07F0F4FEA400C18BFBCF17F4F01
:1047900038BF7047C3F12003994008BF20F00100E3
:1047A000BCF17F4F38BF7047A0F1C04000F007B99F
:1047B0004FEA3C00000A40EBC25028BF1CF0FF0F3C
:1047C0004FEA400CE6D018BFBCF17F4F38BF7047AE
:1047D000EAE79CEA026F05D010EA5C0F08BF00F020
:1047E0000040704710B500F0A4F800BF64FBBE3E67
:1047F000C10DD1F19E0206DB4FEA002343F00043D6
:1048000023FA02F07047004207D54FEA4001B1F1A8
:10481000FE4F02D24FF00000704710B500F089F84B
:1048200049922480002070476FEA20007047000002
:104830004FF47F0C1CEAD0121EBF1CEAD11392EA7F
:104840000C0F93EA0C0F00F0478090EA010F48BF6D
:1048500042F480724FF0004C4CEA00204CEA0121F7
:1048600002EB0302A0FB0113A2F50002002918BF0E
:1048700043F001035B0028BF4FEA330342EB2242BF
:104880005FEA132C4CEBC2502EBFBCEB436FB2F56A
:104890007C0F70474FEA036CBCF1004F08BF20F05B
:1048A0000100B2F57C0F38BF70470BD582F0FF02D4
:1048B00012F5803FC8BF704700F1C040D8BF00F07C
:1048C0000040704700F5000C5FEA4C0C48BF704791
:1048D000B0F1C04000F073B890EA010F0CEAD113B8
:1048E00048BF42F48072624538BF634504D280EA13
:1048F000010000F00040704710B500F01AF800BF4A
:104900008900013E00F007B800F009B85FEA410CE9
:104910005FEA1C6C08D080EA010000F050B85FEA42
:10492000400C5FEA1C6CF6D14FF00040A0F580000F
:1049300070470EF1020E2EF0030E5EF8044B244277
:1049400004D44FEA4102B2F17F4F11D84FEA40033D
:10495000B3F17F4F0CD80ED14FEAD07CB2F17F4F2C
:104960000CEB4C0C0CF1020C08BF4CEBD17C04E0BE
:104970004FF0080C01E04FEAD17C0CEB4C0324FA19
:1049800003F404F00704B4F1040C06D20EEB840C1B
:10499000BDE810404CF0010C6047DFE80CF0070860
:1049A00002024FF00040A0F5800010BD0846420012
:1049B00018BFD2F1807288BF00F0004010BDFF2107
:1049C00041EAD050C005704790EA010F48BF81F01E
:1049D00000413FF5B2AE421A04D882F00042A0EB8B
:1049E000020011444FEAD0524FF07F4C1CEA410FB5
:1049F000A2EBD15318BF9CEA026F4AD04FF0004C93
:104A00004CEA00204CEA012121FA03FCB0EB0C0C2B
:104A10000FD412F0FE0F36D05FEA4C001DD5001205
:104A200040EBC25038BF70471CF03F0F18BF7047B3
:104A30000BE0A2F101025FEA1C2040EBC25038BF3C
:104A400070471CF07F0F18BF7047C3F120039940D7
:104A500014BF401E20F00100704780084FEA122367
:104A600008BF7047B0FA80FCA2EB0C02CCF1280C16
:104A700060FA0CF093EA122F04BF00EBC2507047AB
:104A80004FEAC3707047130A5FEADC1008BF704733
:104A9000F6E79CEA026F04D010EA5C0F08BF002022
:104AA000704710B5FFF745FF40DFF63E81F000404C
:104AB00070470000CC4F000800000000000000001C
:104AC00000000000000000000002000018000000CC
:104AD00000000000000000000000040506070809AF
:104AE00000000000000D0102030405060708090A82
:104AF0000B0C0D0E0F100000000000000000010262
:104B00000304060708090000000001020304000076
:104B1000D84F000800000000000000000000000066
:104B20000000000000040000300000000000000051
:104B300000000000E44F000800000000000000003A
:104B40000000000000000000000200003000000033
:104B50000000000000000000000000000000000055
:104B6000000000000000040404040400000400002D
:104B700014140A00000000000000000000000A0AEF
:104B80001F0A0A1F0A0A000000040E1505060C146D
:104B9000150E0400000012150D152E2C2A1200000F
:104BA0000000040A0A361515291600000202010049
:104BB00000000000000000001008080404040404C1
:104BC0000808100002040408080808080404020089
:104BD00000000004150E0E1504000000000000087F
:104BE000083E08080000000000000000000000006F
:104BF0000202010000000000003F00000000000071
:104C00000000000000000000000200000020101062
:104C1000080804040202010000000E111111111114
:104C2000110E00000000040604040404040E000039
:104C300000000E1111080402011F000000000E11F7
:104C4000100C1010110E00000000080C0C0A091FB7
:104C5000081C000000001F01010F1110110E0000C0
:104C600000000C12010D1311110E000000001E10A7
:104C7000080804040404000000000E11110E1111B4
:104C8000110E000000000E11111916100906000087
:104C9000000000000400000000040000000000000C
:104CA00000040000000404000000100804020204D4
:104CB00008100000000000003F003F00000000005E
:104CC00000000204081010080402000000000E1189
:104CD000110804040004000000001C22292D2D1DD1
:104CE000221C0000000004040C0A0A1E12330000FB
:104CF00000000F12120E1212120F000000001E11FF
:104D000001010101110E000000000F121212121217
:104D1000120F000000001F120A0E0A02121F0000EC
:104D200000001F120A0E0A020207000000001C12F7
:104D300001013911120C000000003312121E121270
:104D40001233000000001F0404040404041F0000C8
:104D500000003E0808080808080809070000371284
:104D60000A060A12123700000000070202020202BD
:104D7000223F000000003B1B1B1B151515350000D2
:104D800000003B1216161A1A1217000000000E112E
:104D900011111111110E000000000F12120E02026B
:104DA0000207000000000E1111111117190E180052
:104DB00000000F12120E0A121237000000001E111E
:104DC00001060810110F000000001F150404040460
:104DD000040E00000000331212121212120C000016
:104DE00000003312120A0A0C04040000000015151A
:104DF00015150E0A0A0A000000001B0A0A04040A1C
:104E00000A1B000000001B0A0A0A0404040E00002A
:104E100000001F0908040402121F00001C040404FF
:104E20000404040404041C0000020204040408082E
:104E3000081010000E0808080808080808080E00E6
:104E4000040A000000000000000000000000000054
:104E5000000000000000003F02040000000000000D
:104E60000000000000000000000C121C123C0000BA
:104E700000030202020E1212120E000000000000D7
:104E8000001C1202120C000000181010101C12124C
:104E9000123C000000000000000C121E021C00006A
:104EA00000182404041E0404041E00000000000076
:104EB000003C120C021C221C00030202020E121201
:104EC000123700000004040000060404040E000071
:104ED00000080800000C0808080808070003020280
:104EE000021A0A060A13000000070404040404045A
:104EF000041F000000000000000F1515151500002C
:104F000000000000000F1212123700000000000025
:104F1000000C1212120C000000000000000F121210
:104F2000120E020700000000001C1212121C1038A2
:104F300000000000001B0602020700000000000045
:104F4000001E020C101E000000000004041E0404D9
:104F5000041C000000000000001B1212123C0000A4
:104F600000000000001B0A0A04040000000000000A
:104F70000015150E0A0A000000000000001B0A04BC
:104F80000A1B000000000000003312120C0804038A
:104F900000000000001E0804041E00001808080895
:104FA000080C080808081800080808080808080875
:104FB000080808080604040404080404040406009D
:104FC0001609000000000000000000006465666132
:104FD000756C745461736B005461736B5F496E69D7
:104FE000740000005461736B5F4D6F6E69746F7273
:104FF000000000001450000800000020A000000085
:105000008C010008B4500008A0000020C02400005B
:10501000A8010008000000000000000000000000DF
:1050200001000000100000000000000000127A00E3
:105030000000000000000000000000000000000070
:105040000000000000000000000000000000000060
:105050000000000000000000000000000000000050
:105060000000000000000000000000000000000040
:105070000000000000000000000000000000000030
:105080000000000000000000000000000000000020
:105090000000000000000000000000000000000010
:1050A0000000000000000000AAAAAAAA0000000058
:0450B00000000000FC
:04000005080001519D
:00000001FF
